:100000000C945D000C9485000C9485000C94850084
:100010000C9485000C9485000C9485000C9485004C
:100020000C9485000C9485000C9485000C9485003C
:100030000C9485000C9485000C9485000C9485002C
:100040000C94AC170C9485000C941C180C94F617A7
:100050000C9485000C9485000C9485000C9485000C
:100060000C9485000C94850000000008000201003B
:100070000003040700000000000000000000000072
:10008000250028002B0000000000240027002A0083
:10009000040404040404040402020202020203032E
:1000A0000303030301020408102040800102040836
:1000B00010200102040810204E1811241FBECFEF9B
:1000C000D8E0DEBFCDBF12E0A0E0B1E0EEE5FEE398
:1000D00002C005900D92AE33B107D9F722E0AEE32E
:1000E000B2E001C01D92A73FB207E1F710E0CDE5F5
:1000F000D0E004C02197FE010E94FA1DCC35D10743
:10010000C9F70E9487180C942D1F0C940000EF92E1
:10011000FF920F931F93CF93DF938B01EA01E88146
:10012000F981E284F384DB01ED91FC910680F78193
:10013000E02D61E070E0C8010995482F61E070E0B2
:10014000CE01F7010995E881F981E484F584D801AD
:10015000ED91FC910084F185E02D61E070E0C80133
:100160000995482F61E070E0CE01F7010995E8811B
:10017000F981E284F384D801ED91FC910680F78146
:10018000E02D62E070E0C8010995482F62E070E060
:10019000CE01F7010995E881F981E484F584D8015D
:1001A000ED91FC910084F185E02D62E070E0C801E2
:1001B0000995482F62E070E0CE01F7010995E881CA
:1001C000F981E688F788D801ED91FC910284F385E6
:1001D000E02D64E070E0C8010995482F64E070E00C
:1001E000CE01F7010995E881F981E688F788D80101
:1001F000ED91FC910284F385E02D6CE070E0C80184
:100200000995482F6CE070E0CE01F7010995E8816F
:10021000F981E688F788D801ED91FC910284F38595
:10022000E02D63E070E0C8010995482F61E070E0BF
:10023000CE01F7010995E881F981E688F788D801B0
:10024000ED91FC910284F385E02D61E070E0C8013E
:100250000995482F62E070E0CE01F7010995E88129
:10026000F981E688F788D801ED91FC910284F38545
:10027000E02D62E070E0C8010995482F63E070E06E
:10028000CE01F7010995E881F981E688F788D80160
:10029000ED91FC910284F385E02D60E070E0C801EF
:1002A0000995482F60E070E0CE01F7010995E881DB
:1002B000F981E688F788D801ED91FC910284F385F5
:1002C000E02D6DE070E0C8010995482F6DE070E009
:1002D000CE01F7010995E881F981E688F788D80110
:1002E000ED91FC910284F385E02D6EE070E0C80191
:1002F0000995482F6EE070E0CE01F7010995E8817D
:10030000F981E688F788D801ED91FC910284F385A4
:10031000E02D6BE070E0C8010995482F6BE070E0BC
:10032000CE01F7010995E881F981E688F788D801BF
:10033000ED91FC910284F385E02D6AE070E0C80144
:100340000995482F6AE070E0CE01F7010995E88130
:10035000F981E688F788D801ED91FC910284F38554
:10036000E02D68E070E0C8010995482F68E070E072
:10037000CE01F7010995E881F981E688F788D8016F
:10038000ED91FC910284F385E02D69E070E0C801F5
:100390000995482F69E070E0CE01F701DF91CF9118
:1003A0001F910F91FF90EF900994EF92FF920F939E
:1003B0001F93CF93DF938B01EA01E881F981E284F7
:1003C000F384DB01ED91FC910680F781E02D61E083
:1003D00070E0C8010995482F61E070E0CE01F70197
:1003E0000995E881F981E484F584D801ED91FC91C7
:1003F0000084F185E02D61E070E0C8010995482F87
:1004000061E070E0CE01F7010995E881F981E284AD
:10041000F384D801ED91FC910680F781E02D62E034
:1004200070E0C8010995482F62E070E0CE01F70145
:100430000995E881F981E484F584D801ED91FC9176
:100440000084F185E02D62E070E0C8010995482F35
:1004500062E070E0CE01F7010995E881F981E68854
:10046000F788D801ED91FC910284F385E02D64E0DA
:1004700070E0C8010995482F64E070E0CE01F701F3
:100480000995E881F981E688F788D801ED91FC911A
:100490000284F385E02D6CE070E0C8010995482FD7
:1004A0006CE070E0CE01F7010995E881F981E688FA
:1004B000F788D801ED91FC910284F385E02D60E08E
:1004C00070E0C8010995482F61E070E0CE01F701A6
:1004D0000995E881F981E688F788D801ED91FC91CA
:1004E0000284F385E02D63E070E0C8010995482F90
:1004F00062E070E0CE01F7010995E881F981E688B4
:10050000F788D801ED91FC910284F385E02D61E03C
:1005100070E0C8010995482F63E070E0CE01F70153
:100520000995E881F981E688F788D801ED91FC9179
:100530000284F385E02D62E070E0C8010995482F40
:1005400060E070E0CE01F7010995E881F981E68865
:10055000F788D801ED91FC910284F385E02D6DE0E0
:1005600070E0C8010995482F6DE070E0CE01F701F9
:100570000995E881F981E688F788D801ED91FC9129
:100580000284F385E02D6EE070E0C8010995482FE4
:100590006EE070E0CE01F7010995E881F981E68807
:1005A000F788D801ED91FC910284F385E02D6BE092
:1005B00070E0C8010995482F6BE070E0CE01F701AB
:1005C0000995E881F981E688F788D801ED91FC91D9
:1005D0000284F385E02D6AE070E0C8010995482F98
:1005E0006AE070E0CE01F7010995E881F981E688BB
:1005F000F788D801ED91FC910284F385E02D68E045
:1006000070E0C8010995482F68E070E0CE01F7015D
:100610000995E881F981E688F788D801ED91FC9188
:100620000284F385E02D69E070E0C8010995482F48
:1006300069E070E0CE01F701DF91CF911F910F913A
:10064000FF90EF900994EF92FF920F931F93CF9337
:10065000DF938B01EA01E881F981E284F384DB0115
:10066000ED91FC910680F781E02D61E070E0C8011A
:100670000995482F61E070E0CE01F7010995E88106
:10068000F981E484F584D801ED91FC910084F18531
:10069000E02D61E070E0C8010995482F61E070E04D
:1006A000CE01F7010995E881F981E284F384D8014C
:1006B000ED91FC910680F781E02D62E070E0C801C9
:1006C0000995482F62E070E0CE01F7010995E881B5
:1006D000F981E484F584D801ED91FC910084F185E1
:1006E000E02D62E070E0C8010995482F62E070E0FB
:1006F000CE01F7010995E881F981E688F788D801EC
:10070000ED91FC910284F385E02D64E070E0C80176
:100710000995482F64E070E0CE01F7010995E88162
:10072000F981E688F788D801ED91FC910284F38580
:10073000E02D6CE070E0C8010995482F6CE070E096
:10074000CE01F7010995E881F981E688F788D8019B
:10075000ED91FC910284F385E02D61E070E0C80129
:100760000995482F61E070E0CE01F7010995E88115
:10077000F981E688F788D801ED91FC910284F38530
:10078000E02D62E070E0C8010995482F62E070E05A
:10079000CE01F7010995E881F981E688F788D8014B
:1007A000ED91FC910284F385E02D63E070E0C801D7
:1007B0000995482F63E070E0CE01F7010995E881C3
:1007C000F981E688F788D801ED91FC910284F385E0
:1007D000E02D60E070E0C8010995482F60E070E00E
:1007E000CE01F7010995E881F981E688F788D801FB
:1007F000ED91FC910284F385E02D6DE070E0C8017D
:100800000995482F6DE070E0CE01F7010995E88168
:10081000F981E688F788D801ED91FC910284F3858F
:10082000E02D6EE070E0C8010995482F6EE070E0A1
:10083000CE01F7010995E881F981E688F788D801AA
:10084000ED91FC910284F385E02D6BE070E0C8012E
:100850000995482F6BE070E0CE01F7010995E8811A
:10086000F981E688F788D801ED91FC910284F3853F
:10087000E02D6AE070E0C8010995482F6AE070E059
:10088000CE01F7010995E881F981E688F788D8015A
:10089000ED91FC910284F385E02D68E070E0C801E1
:1008A0000995482F68E070E0CE01F7010995E881CD
:1008B000F981E688F788D801ED91FC910284F385EF
:1008C000E02D69E070E0C8010995482F69E070E00B
:1008D000CE01F701DF91CF911F910F91FF90EF9023
:1008E0000994EF92FF920F931F93CF93DF938B01A5
:1008F000EA01E881F981E284F384DB01ED91FC9166
:100900000680F781E02D60E070E0C8010995482F6E
:1009100060E070E0CE01F7010995E881F981E48497
:10092000F584D801ED91FC910084F185E02D60E023
:1009300070E0C8010995482F60E070E0CE01F70132
:10094000DF91CF911F910F91FF90EF9009944F92FB
:100950005F926F927F92AF92BF92CF92DF92EF92AF
:10096000FF920F931F93CF93DF93EB018A01DA017C
:10097000ED91FC91E284F384E881F9810680F781AE
:10098000E02D61E070E0CE010995482F61E070E054
:10099000C801F7010995D801ED91FC91E484F58433
:1009A000E881F9810084F185E02D61E070E0CE01FD
:1009B0000995482F61E070E0C801F7010995E881C9
:1009C000F9810680F781E02D62E070E0CE010995A3
:1009D000682F880F770B60587F4F072E000C880B0D
:1009E000990B0E94B01C20E030E045E553E40E94E2
:1009F000651D20E030E044E752E40E94061C6B01D4
:100A00007C01E881F9810084F185E02D62E070E0ED
:100A1000CE010995682F880F770B60587F4F072EFE
:100A2000000C880B990B0E94B01C20E030E045E5DB
:100A300053E40E94651D20E030E044E752E40E9448
:100A4000061C2B013C01D801ED91FC91A284B384DA
:100A500020E030E04FE753E4C701B6010E94601D7B
:100A6000181664F020E030E040E053E4C701B6011E
:100A70000E94941B0E94781C462F01C04FE762E041
:100A800070E0C801F5010995D801ED91FC91E4846D
:100A9000F58420E030E04FE753E4C301B2010E9447
:100AA000601D181664F020E030E040E053E4C3011C
:100AB000B2010E94941B0E94781C462F01C04FE790
:100AC00062E070E0C801F7010995D801ED91FC9151
:100AD000E688F788E881F9810284F385E02D64E0F7
:100AE00070E0CE010995482F64E070E0C801F7017D
:100AF0000995D801ED91FC91E688F788E881F981A4
:100B00000284F385E02D6CE070E0CE010995482F5A
:100B10006CE070E0C801F7010995D801ED91FC91F6
:100B2000E688F788E881F9810284F385E02D61E0A9
:100B300070E0CE010995482F61E070E0C801F7012F
:100B40000995D801ED91FC91E688F788E881F98153
:100B50000284F385E02D62E070E0CE010995482F14
:100B600062E070E0C801F7010995D801ED91FC91B0
:100B7000E688F788E881F9810284F385E02D63E057
:100B800070E0CE010995482F63E070E0C801F701DD
:100B90000995D801ED91FC91E688F788E881F98103
:100BA0000284F385E02D60E070E0CE010995482FC6
:100BB00060E070E0C801F7010995D801ED91FC9162
:100BC000E688F788E881F9810084F185E02D62E00C
:100BD00070E0CE010995D82EE881F9810284F38571
:100BE000E02D6DE070E0CE01099541E0BDEBDB1634
:100BF0000CF440E0482B6DE070E0C801F701099566
:100C0000D801ED91FC91E688F788E881F9810680AA
:100C1000F781E02D62E070E0CE010995D82EE881E1
:100C2000F9810284F385E02D6EE070E0CE01099534
:100C300041E0BDEBDB160CF440E0482B6EE070E0C9
:100C4000C801F7010995D801ED91FC91E688F78874
:100C5000E881F9810284F385E02D6BE070E0CE013C
:100C60000995482F6BE070E0C801F7010995D8019C
:100C7000ED91FC91E688F788E881F9810284F3859B
:100C8000E02D6AE070E0CE010995482F6AE070E03F
:100C9000C801F7010995D801ED91FC91E688F78824
:100CA000E881F9810284F385E02D68E070E0CE01EF
:100CB0000995482F68E070E0C801F7010995D8014F
:100CC000ED91FC91E688F788E881F9810284F3854B
:100CD000E02D69E070E0CE010995482F69E070E0F1
:100CE000C801F701DF91CF911F910F91FF90EF9015
:100CF000DF90CF90BF90AF907F906F905F904F90BC
:100D000009940F931F93CF938C01C62F0E947E1BD3
:100D1000C81721F06C2FC8010E94861B8C2FCF9121
:100D20001F910F910895FC01918D228D892F90E0E4
:100D3000805C9F4F821B91098F739927089580E0F3
:100D400090E0892B29F00E94331781110C94000048
:100D50000895DC01ED91FC910284F385E02D6DE0B6
:100D600070E00994FC0197859F7121F490899F7729
:100D700081E009F080E00895FC0197859F719D3026
:100D800029F490899F7781E0903509F080E00895FB
:100D90009B0177FF02C0295F3F4F43E035952795C0
:100DA0004A95E1F7FC01E20FF31F278530E0CB0104
:100DB00068E070E00E94D21DA90102C055954795D8
:100DC0008A95E2F7CA0181700895660F771F860F32
:100DD000971FFC01828980580895660F771F860F40
:100DE000971FFC01818980580895FC0114A608957D
:100DF000FC0184A50895860F971F4195FC0141874A
:100E00000895860F971FFC01418708959B01442395
:100E1000E9F077FF02C0295F3F4F53E035952795F2
:100E20005A95E1F7FC01E20FF31FCB0168E070E097
:100E30000E94D21D21E030E0A90102C0440F551FDD
:100E40008A95E2F7CA019381892B1DC077FF02C002
:100E5000295F3F4F43E0359527954A95E1F7FC011F
:100E6000E20FF31FCB0168E070E00E94D21D21E089
:100E700030E0A90102C0440F551F8A95E2F7CA016C
:100E800080959381892383830895660F771FFC01E2
:100E9000E60FF71F8FE7489F402D112440584683E7
:100EA00008956F5F7F4F660F771FFC01E60FF71FF6
:100EB0008FE7489F402D1124405843830895660FC3
:100EC000771F860F971F4058FC01468308956F5F78
:100ED0007F4F660F771F860F971F4058FC01438393
:100EE0000895FC01138280E8848385838683878349
:100EF0008087118612860895CF92DF92EF92FF923B
:100F00000F931F93CF93DF938C01EB017A01DC01E8
:100F100015968D919C9116978130910521F002973D
:100F200009F45DC014C0E881F9810088F189E02DE1
:100F3000CB010995882331F082E090E0F801968397
:100F40008583C3C1D80116961C921E921597D701AE
:100F5000ED91FC91C284D384E881F9810680F78108
:100F6000E02D60E070E0CE010995682F880F770BC7
:100F7000880B990B0E94B01CAB01BC01C8010E94F8
:100F80007211482F60E070E0C701F6010995D701A2
:100F9000ED91FC91C484D584E881F9810084F185C8
:100FA000E02D60E070E0CE010995682F880F770B87
:100FB000880B990B0E94B01CAB01BC01C8010E94B8
:100FC0007211482F60E070E0C701F601DF91CF9108
:100FD0001F910F91FF90EF90DF90CF900994D8016F
:100FE0001396ED91FC9114973496EE0FFF1FE00FCE
:100FF000F11F4081518157FF02C04F5F5F4F5595F0
:101000004795D701ED91FC910284F385E02D60E0D6
:1010100070E0C7010995D8011396ED91FC911497E2
:101020003896EE0FFF1FE00FF11F4081518157FFEF
:1010300002C04F5F5F4F55954795D701ED91FC91E9
:101040000484F585E02D60E070E0C7010995E88132
:10105000F9810088F189E02DCE010995882309F4F2
:101060004DC1F8018781E881F9810284F385E02D83
:10107000882309F461C062E070E0CE010995811116
:1010800074C1E881F9810284F385E02D63E070E0AA
:10109000CE010995811169C1E881F9810284F38546
:1010A000E02D61E070E0CE01099581115EC1E8811B
:1010B000F9810284F385E02D60E070E0CE010995AE
:1010C000811153C1E881F9810284F385E02D68E044
:1010D00070E0CE010995811148C1E881F98102844F
:1010E000F385E02D69E070E0CE01099581113DC1E5
:1010F000E881F9810284F385E02D6AE070E0CE0199
:101100000995811132C1E881F9810284F385E02DCE
:101110006BE070E0CE010995811127C1E881F9816A
:101120000284F385E02D64E070E0CE010995811121
:101130001CC1F801178219C163E070E0CE01099566
:101140008823C1F0D8011396ED91FC911497EE0F0E
:10115000FF1FE00FF11F808591858230910514F00B
:10116000019702C081E090E09187808781E0F801DB
:101170008783FBC0E881F9810284F385E02D62E07A
:1011800070E0CE0109958823A1F0D8011396ED9166
:10119000FC911497EE0FFF1FE00FF11F20853185A2
:1011A00080899189019728173907F4F6C9010196BA
:1011B000DBCFE881F9810284F385E02D61E070E006
:1011C000CE0109958823A1F0D8011396ED91FC91E9
:1011D0001497EE0FFF1FE00FF11F208931898085E2
:1011E000918501968217930704F5C90101971DC0E7
:1011F000E881F9810284F385E02D60E070E0CE01A2
:1012000009958823A9F0D8011396ED91FC911497C4
:10121000EE0FFF1FE00FF11F808991898F3F91052D
:1012200014F4019602C08FEF90E0918B808B9ECFDB
:10123000E881F9810284F385E02D64E070E0CE015D
:101240000995882381F0D8011396ED91FC911497AC
:10125000EE0FFF1FE00FF11F118610868FE790E061
:10126000918B808B47C0E881F9810284F385E02D62
:101270006BE070E0CE010995882321F0F80114821B
:10128000138223C0E881F9810284F385E02D68E0B0
:1012900070E0CE010995882341F081E090E0D8010B
:1012A00014969C938E93139726C0E881F98102844B
:1012B000F385E02D6AE070E0CE010995882339F0CE
:1012C00082E090E0F8019483838381E051CFE8814C
:1012D000F9810284F385E02D69E070E0CE01099583
:1012E000882309F442C083E090E0D80114969C93CF
:1012F0008E93139781E017968C9337C08091E30209
:101300009091E402892B61F17801B8E0EB0EF11CB9
:10131000C0E0D0E0F7016081F2E0EF0EF11C8091B7
:10132000E3029091E4028C0F9D1F0E948106809140
:10133000E3029091E4028C0F9D1FD70116966C91E9
:1013400001960E9481062296C830D10519F7809136
:10135000E3029091E402F801638108960E948106FD
:10136000D80116961C921E921597DF91CF911F916E
:101370000F91FF90EF90DF90CF9008956F927F9242
:101380008F929F92AF92BF92CF92DF92EF92FF9295
:101390000F931F93CF93DF9300D000D0CDB7DEB76C
:1013A0008C01DC0191968C9191978111E1C088E0CC
:1013B000E8E1F1E01F9601900D928A95E1F7D801DE
:1013C000AE58BF4F80E090E067E070E041E050E051
:1013D0009C0127703327FB01E21BF30B3A0102C08B
:1013E000660C771CEA95E2F79301FC0133E0F59572
:1013F000E7953A95E1F7E00FF11F378523232D9309
:1014000001968034910521F7780162E2E60EF11C25
:1014100080E4D7011D928A95E9F71C8261E0CE0134
:1014200004960E9482106AE070E0C7010E942D11AC
:10143000C8018E549F4F2AE0FC0111922A95E9F7CA
:101440004701F70140E050E077E0C72ED12CA19191
:101450009A0163E0359527956A95E1F7200F311FD2
:10146000590162EBA60EB11C61E070E0A11102C04F
:1014700060E070E0DA01A770BB2736016A1A7B0AC8
:1014800001C0660F6A94EAF7D901AE54BF4F2C91A0
:10149000622BD5016C934F5F5F4F40355105B9F614
:1014A000FC01208121110AC0F801ED54FF4F208179
:1014B000211104C031962081222329F081E0D80136
:1014C00091968C9306C04AE050E060E071E00E9483
:1014D000261F8AE0E3EFF1E0D801579601900D92C4
:1014E0008A95E1F780E5F70111928A95E9F781E4A1
:1014F000898361E0CE0101960E9482106AE070E06B
:10150000C7010E942D11019779F58AE0F8017796BD
:10151000DF011D928A95E9F720E030E047E050E0D6
:10152000F40161914F01F90193E0F595E7959A95E2
:10153000E1F7E00FF11F81E090E0611102C080E06F
:1015400090E0B901677077273A01661A770A01C0FF
:10155000880F6A94EAF79789892B878B2F5F3F4F13
:1015600020353105E9F6BDC0D80191961C92B9C06D
:101570007801B2E2EB0EF11C80E4F70111928A953A
:10158000E9F7D8011896ED91FC91199782818111A4
:1015900003C0EAE0F1E002C0EDE0F1E0808191817A
:1015A000A28189839A83AB8363E0CE0101960E9476
:1015B000821068E070E0C7010E942D11F80182A539
:1015C000882309F48CC020E4F701C8018E589F4F8E
:1015D000DC0101900D922A95E1F728E0F8013F9691
:1015E000DF011D922A95E9F7DC0120E030E047E0B9
:1015F00050E06D91F90183E0F595E7958A95E1F763
:10160000E00FF11F81E090E0611102C080E090E006
:10161000B901677077273A01661A770A01C0880F07
:101620006A94EAF79785892B87872F5F3F4F20348D
:101630003105F9F665EF71E0F80120E030E0DB01FB
:101640005D91BD01818990E0418D450F841B910919
:1016500047FD939597FD07C08F3F910529F024F032
:101660008FEF90E001C080E0818BA8014E575F4F63
:10167000982F9078DA019C934F5F5F4F982F90746A
:10168000DA019C934F5F5F4F982F9072DA019C9321
:101690004F5F5F4F982F9071DA019C934F5F5F4FC0
:1016A000982F9870DA019C934F5F5F4F982F94703A
:1016B000DA019C934F5F5F4F982F9270DA019C93F1
:1016C0004F5F5F4F8170DA018C932F5F3F4F3196F0
:1016D000085F1F4F2630310509F0B1CF02C0F80175
:1016E00011A20F900F900F900F90DF91CF911F914B
:1016F0000F91FF90EF90DF90CF90BF90AF909F90B1
:101700008F907F906F9008950C94981EEF92FF92A7
:101710000F931F93CF93DF93CDB7DEB728970FB604
:10172000F894DEBF0FBECDBF8C01FC01E85BFE4F1D
:101730008081833440F4813408F05CC0882331F028
:10174000803411F16AC08F3F09F067C089E0F80169
:101750008383148283E0858380E8868317821086E2
:1017600011861286FF24F394F386F48640E063E04A
:10177000C80103960E94450FF801F4A660E070E0EE
:10178000C8010E94FA0F49C080913E0298012C5D69
:101790003F4F790181110CC028E0C8010396FC017C
:1017A000D70101900D922A95E1F741E068E00CC065
:1017B00088E0F901DE01119601900D928A95E1F71A
:1017C00041E068E0CE0101960E94450FF801EF2844
:1017D00011F4128207C0E65BFE4F80818170808326
:1017E000F801828361E070E0C8010E94FA0F8093E3
:1017F0003E0213C0F801138280E8848385838683C8
:10180000878380871186128681E08387848741E001
:101810006AE0C80103960E94450F28960FB6F89417
:10182000DEBF0FBECDBFDF91CF911F910F91FF9013
:10183000EF90089560E070E00C94FA0FFC01848D45
:10184000DF01A80FB11DA35ABF4F2C91848D90E0EA
:1018500001968F739927848FA689B7892C93A089C5
:10186000B1898C91837080648C93938D848D98134F
:1018700006C00288F389E02D80818F7D80830895E2
:10188000CF92DF92EF92FF920F931F93CF93DF934C
:10189000EC011A8284E291E0998388831C821B8286
:1018A000198618868FE790E0998B888B1B861A869D
:1018B0009B8B8A8B1D861C869D8B8C8B1F861E8620
:1018C0009F8B8E8B0091E3021091E40201151105AC
:1018D00009F05DC082E00E94840D8C019093E402C7
:1018E0008093E302009779F569E070E082E00E945E
:1018F000F90C9093E4028093E302892B09F46BC006
:1019000000E010E08091E3029091E40260E0800F3B
:10191000911F0E9481068091E3029091E402800F62
:10192000911F6FE701960E9481060E5F1F4F0830DE
:10193000110541F78091E3029091E40260E008967E
:101940000E94810648C008960E947E1B90E09C83FE
:101950008B837E0188E0E80EF11C6E01E0E1CE0E83
:10196000D11CC8010E947E1B90E0F70181939193E6
:101970007F01C80101960E947E1B90E0F7019783CA
:1019800086830E5F1F4FCE14DF0459F724C0C801B1
:1019900008960E947E1B90E09C838B837E01F8E07A
:1019A000EF0EF11C6E0180E1C80ED11CC8010E942F
:1019B0007E1B90E0F701819391937F01C80101960E
:1019C0000E947E1B90E0F701978386830E5F1F4F76
:1019D000EC14FD0459F781E090E09E838D83DF9144
:1019E000CF911F910F91FF90EF90DF90CF900895CE
:1019F00008958F929F92AF92BF92CF92DF92EF9213
:101A0000FF920F931F93CF93DF93C82E5B01E0905B
:101A10004402F0904502C0E0D0E00AE010E0EC168D
:101A2000FD060CF462C0C8010E947E1B98012E5F67
:101A30003F4F49018F3F21F0EC16FD0609F04CC0E5
:101A4000C4010E947E1BD82EEC16FD0651F090E0DA
:101A50008A159B050CF440C09C2F8D2FE701E92EC1
:101A6000F82E6C2DC8010E94810660E0C801019625
:101A70000E9481060D5F1F4FEC16FD06A1F08D2D13
:101A800090E00297A816B9068CF47801EA0CFB1CCA
:101A90006FEFC7010E9481066D2D6A196350C7015F
:101AA00002960E94810621966A2D01C06D2DC40107
:101AB0000E94810680914402909145028C179D07F7
:101AC00049F0D0934502C09344026C2F81E090E02E
:101AD0000E948106C8010BC0C4010E947E1B90E0D9
:101AE0000396080F191F21969ACF80E090E0DF91AE
:101AF000CF911F910F91FF90EF90DF90CF90BF900B
:101B0000AF909F908F900895DF92EF92FF920F9386
:101B10001F93CF93DF93D82EE0904402F0904502BC
:101B200000E010E0CAE0D0E00E151F05CCF4CE01B5
:101B30000E947E1BD81209C0CE0101960E947E1B16
:101B4000811103C0CE0103960DC0CE0102960E9402
:101B50007E1B90E00396C80FD91F0F5F1F4FE4CF85
:101B600080E090E0DF91CF911F910F91FF90EF9077
:101B7000DF9008950F931F93CF93DF93EC018B01B8
:101B80008E819F81009721F00E94981E1F821E82E5
:101B90008A819B81009711F00E94981E1B830A8303
:101BA000DF91CF911F910F9108952F923F924F9205
:101BB0005F926F927F928F929F92AF92BF92CF92DD
:101BC000DF92EF92FF920F931F93CF93DF93CDB7E6
:101BD000DEB728970FB6F894DEBF0FBECDBF9E8349
:101BE0008D836A017B0120E030E040E053E4C701CF
:101BF000B6010E94601D181654F420E030E040E861
:101C000053E4C701B6010E94941B6B017C0120E0E4
:101C100030E0A901C701B6010E94011C87FF0BC07B
:101C2000F7FAF094F7F8F094812C912C90E8A92E13
:101C30009FEBB92E13C020E030E0A901C701B60127
:101C40000E94011C882339F0812C912C80E8A82E59
:101C50008FE3B82E03C0812C912C5401ED81FE81BD
:101C600027803084B101032C000C880B990B0E9453
:101C7000B01C2B013C01A70196010E94011CED81C3
:101C8000FE8118160CF4B5C001851285B801012E2D
:101C9000000C880B990B0E94B01C69837A838B839C
:101CA0009C83A70196010E94601D18160CF041C08C
:101CB000ED81FE810584F685E02DFA83E983ED81CF
:101CC000FE816385748529813A81621B730B072E1F
:101CD000000C880B990B0E94B01C6D837E838F8350
:101CE0009887A3019201C701B6010E94941B9B0132
:101CF000AC016D817E818F8198850E94651D6B018D
:101D00007C01B80162197309072E000C880B990B2E
:101D10000E94B01C9B01AC01C701B6010E94061CC9
:101D20006B017C01E981FA81BF01FF0F880B990BE0
:101D300040C020E030E04EEF52E4C701B6010E94FF
:101D4000011C87FF3DC0ED81FE81238434846FE751
:101D500070E062197309072E000C880B990B0E9422
:101D6000B01C2B013C0129813A814B815C81C70168
:101D7000B6010E94941B9B01AC01C301B2010E94F9
:101D8000651D6B017C012FE730E0201B310BB90191
:101D9000330F880B990B0E94B01C9B01AC01C7014B
:101DA000B6010E94061C6B017C01B101330C880B4B
:101DB000990B0E94B01C9B01AC01C701B60116C073
:101DC00020E030E04EEF52E4C701B6010E94941BC0
:101DD00020E030E0A9010E94651D20E030E0A9016B
:101DE0000E94061C20E030E04EEF52E40E94951B5A
:101DF00010C065857685072E000C880B990B0E9414
:101E0000B01CA70196010E94651DA30192010E94CA
:101E1000061CA50194010E94651D6B017C0120E058
:101E200030E040E053EC0E94011C87FD10C020E030
:101E300030E04EEF52E4C701B6010E94601D181653
:101E40004CF0C701B6010E94781CCB0105C080E8A8
:101E50009FEF02C08FE790E028960FB6F894DEBFA0
:101E60000FBECDBFDF91CF911F910F91FF90EF90EB
:101E7000DF90CF90BF90AF909F908F907F906F90AA
:101E80005F904F903F902F900895FC0128E0539A67
:101E9000808190E0880F892F881F990B892B09F486
:101EA00030C0000000000000000000000000000042
:101EB0000000539800000000000000000000000037
:101EC0000000000000000000000000000000000012
:101ED0000000000000000000000000000000000002
:101EE00000000000000000000000000000000000F2
:101EF00000000000000000000000000000000000E2
:101F000030C00000000000000000000000000000E1
:101F100000000000000000000000000000000000C1
:101F200000000000000000000000000000000000B1
:101F300000000000000000000000000000000000A1
:101F40000000000000000000000000000000000091
:101F50000000000000000000000000000000000081
:101F60005398215069F000000000000000000000BC
:101F700000000000000000008081880F808387CF70
:101F80000000000000000000615031F0000000007F
:101F90000000000031967ACF000000000000000031
:101FA0000000000000000000539A00000000000044
:101FB0000000000000000000000000000000000021
:101FC0000000000000000000442391F00000000029
:101FD0000000000000000000000000000000000001
:101FE00000000000000000000000000000000000F1
:101FF00053980895CF93DF93DC01FC01E85BFE4F1B
:1020000083E0EF0119928A95E9F7EF01161617069A
:102010009CF484EC99E04B9907C081E09C968C93EA
:102020009C9728E030E01BC00197A9F79C968C9103
:102030009C97882309F461C09C968C919C97811190
:102040000AC080E290E04B9902C080E290E00197E4
:1020500018161906C4F328E030E04B99FECF0000B3
:102060000000000000000000000000000000000070
:102070000000000000000000000000000000000060
:102080000000000000000000000000000000000050
:102090000000000000000000000000000000000040
:1020A000000000000000000000004B9B03C0808186
:1020B000816080832150310931F08081880F8083D5
:1020C0004B9BFECFCACF8881803441F4CD01865B23
:1020D0009E4FE817F90711F03196BDCF4B9BFECF0D
:1020E0008CE090E04B9902C08CE090E001971816CC
:1020F0001906C4F381E090E002C080E090E0DF9137
:10210000CF910895FC0128E08AB180638AB980816B
:1021100090E0880F892F881F990B892B09F432C012
:1021200000000000000000000000000000000000AF
:102130008AB18F7C8AB90000000000000000000016
:10214000000000000000000000000000000000008F
:10215000000000000000000000000000000000007F
:10216000000000000000000000000000000000006F
:10217000000000000000000000000000000000005F
:10218000000032C00000000000000000000000005D
:10219000000000000000000000000000000000003F
:1021A000000000000000000000000000000000002F
:1021B000000000000000000000000000000000001F
:1021C000000000000000000000000000000000000F
:1021D00000000000000000000000000000000000FF
:1021E00000008AB18F7C8AB9215069F0000000009C
:1021F00000000000000000000000000000008081DE
:10220000880F808381CF0000000000000000615033
:1022100031F00000000000000000319674CF000093
:1022200000000000000000000000000000008AB173
:1022300080638AB900000000000000000000000078
:10224000000000000000000000000000000000008E
:1022500000008AB18F7C8AB90895FC01660F660F71
:10226000660F9FE329B1207329F09150D9F780E0E0
:1022700090E0089500000000000000000000000051
:10228000000000000000000000000000000000004E
:10229000000000000000000000000000000000003E
:1022A000000000000000000000000000000000002E
:1022B000000000000000000000000000000000001E
:1022C00099B190739193615051F09FE329B12073BC
:1022D00009F0C7CF9150D1F782E090E0089581E0F6
:1022E00090E008954F925F926F927F928F929F92AB
:1022F000AF92BF92CF92DF92EF92FF92CF93DF9394
:10230000EC016A017B0120E030E040E053E4C701CA
:10231000B6010E94601D181654F420E030E040E839
:1023200053E4C701B6010E94941B6B017C0120E0BD
:1023300030E0A901C701B6010E94011C87FF0BC054
:10234000F7FAF094F7F8F094812C912C40E8A42E41
:102350004FEBB42E13C020E030E0A901C701B60155
:102360000E94011C882339F0812C912C30E8A32E87
:102370003FE3B32E03C0812C912C54018B819C81AF
:10238000880F991FC80FD91F68857985072E000C03
:10239000880B990B0E94B01C2B013C01A7019601F0
:1023A0000E94601D87FF44C0A3019201C701B601CE
:1023B0000E94941B6B017C01A301920160E070E01C
:1023C0008EEF92E40E94941B9B01AC01C701B60101
:1023D0000E94061C6B017C0168897989072E000C1C
:1023E000880B990B0E94B01C9B01AC01C701B60180
:1023F0000E94651DA50194010E94651D6B017C0171
:1024000020E030E040E053EC0E94011C87FD13C047
:1024100020E030E04EEF52E4C701B6010E94601D9B
:10242000181664F0C701B6010E94781CCB0108C0E1
:1024300080E090E005C080E89FEF02C08FE790E069
:10244000DF91CF91FF90EF90DF90CF90BF90AF9052
:102450009F908F907F906F905F904F900895CF9353
:10246000DF9390E0FC01EC55FF4F2491FC01E05715
:10247000FF4F84918823C1F090E0880F991FFC01E1
:10248000EA57FF4FC591D491FC01E458FF4FA59145
:10249000B4919FB7F8948881E22FE0958E238883CA
:1024A0008C91E823EC939FBFDF91CF91089590E04A
:1024B000FC01E859FF4F2491FC01EC55FF4F34918A
:1024C000FC01E057FF4FE491EE23B9F1222339F1EB
:1024D000233091F038F42130A9F0223001F584B591
:1024E0008F7D12C0273091F02830A1F02430B9F44C
:1024F000809180008F7D03C0809180008F778093D2
:1025000080000DC084B58F7784BD09C08091B00074
:102510008F7703C08091B0008F7D8093B000F0E092
:10252000EE0FFF1FE458FF4FA591B4919FB7F894A9
:102530008C91309538233C939FBF0895682F86E493
:1025400092E00C943D173FB7F89480913F02909130
:102550004002A0914102B091420226B5A89B05C05D
:102560002F3F19F00196A11DB11D3FBFBA2FA92F12
:10257000982F8827820F911DA11DB11DBC01CD018F
:1025800042E0660F771F881F991F4A95D1F708957B
:102590002091E7023091E8022115310529F0682FDA
:1025A000C90101960C9481060895682F8091E70275
:1025B0009091E802009711F00C9481060895DF9243
:1025C000EF92FF920F931F93CF93DF93EC018B0158
:1025D0007A018C819D818130910521F0029709F467
:1025E00071C011C0DB01ED91FC910088F189E02DF3
:1025F000CB010995882329F082E090E09D838C83AC
:10260000DDC11D821C82D801ED91FC910680F7810D
:10261000E02D60E070E0C8010995D801ED91FC91D2
:102620000084F185E02D60E070E0C8010995D801D3
:10263000ED91FC910680F781E02D60E070E0C8012B
:102640000995682F880F770B880B990B0E94B01C97
:10265000AB01BC01CE010E94D50DD82ED801ED9161
:10266000FC910084F185E02D60E070E0C8010995DF
:10267000682F880F770B880B990B0E94B01CAB0159
:10268000BC01CE010E94D50DC82FD701ED91FC9160
:102690000284F385E02D4D2D60E070E0C7010995BF
:1026A000D701ED91FC910484F585E02D4C2F60E07D
:1026B00070E0C701DF91CF911F910F91FF90EF90D4
:1026C000DF900994AF81B885A25CBE4FFA0180818A
:1026D0009181FC01228533854C9160E070E0C70157
:1026E000F9010995A985BA85A25CBE4FF7018081E1
:1026F0009181FC01248535854C9160E070E0C70133
:10270000F9010995D801ED91FC910088F189E02D3E
:10271000C8010995882309F454C18E81D801ED912F
:10272000FC910284F385E02D882309F468C062E0FF
:1027300070E0C801099581115FC1D801ED91FC914C
:102740000284F385E02D63E070E0C80109958111F2
:1027500053C1D801ED91FC910284F385E02D61E035
:1027600070E0C8010995811147C1D801ED91FC9134
:102770000284F385E02D60E070E0C80109958111C5
:102780003BC1D801ED91FC910284F385E02D68E016
:1027900070E0C801099581112FC1D801ED91FC911C
:1027A0000284F385E02D69E070E0C801099581118C
:1027B00023C1D801ED91FC910284F385E02D6AE0FC
:1027C00070E0C8010995811117C1D801ED91FC9104
:1027D0000284F385E02D6CE070E0C8010995811159
:1027E0000BC1D801ED91FC910284F385E02D64E0EA
:1027F00070E0C80109958111FFC01E82FDC063E031
:1028000070E0C8010995882351F08F819885823046
:10281000910514F0019719C081E090E016C0D8012D
:10282000ED91FC910284F385E02D62E070E0C80137
:102830000995882369F02F81388589859A850197C4
:102840002817390714F4C901019698878F83B6C0F9
:10285000D801ED91FC910284F385E02D61E070E0F8
:10286000C8010995882361F029853A858F8198856B
:102870000196821793070CF051C0C90101974EC011
:10288000D801ED91FC910284F385E02D60E070E0C9
:10289000C8010995882351F089859A858E3791055D
:1028A00014F401963BC08EE790E038C0D801ED915A
:1028B000FC910284F385E02D64E070E0C801099585
:1028C0008823D1F08B81813049F0823071F087E12B
:1028D00090E098878F8385E290E020C084E190E0CB
:1028E00098878F8380E290E019C08EE190E098870E
:1028F0008F8389E290E012C0D801ED91FC910284AF
:10290000F385E02D6CE070E0C8010995882349F05B
:1029100088E090E098878F838AE290E09A878987A1
:102920004DC0D801ED91FC910284F385E02D68E063
:1029300070E0C8010995882369F082E08B838EE1FD
:1029400090E09E878D8789E290E09C878B8789E461
:1029500090E032C0D801ED91FC910284F385E02D26
:102960006AE070E0C8010995882379F081E08B83E3
:1029700024E130E03E872D8720E230E03C872B8742
:1029800025E330E0388B2F871AC0D801ED91FC91F8
:102990000284F385E02D69E070E0C8010995882381
:1029A00059F11B8287E190E09E878D8785E290E058
:1029B0009C878B8787E490E0988B8F8781E08E835C
:1029C0001BC08091E5029091E602009799F06F811B
:1029D0000E9481068091E5029091E6026985019648
:1029E0000E9481068091E5029091E6026B81029639
:1029F0000E9481061D821C82DF91CF911F910F9151
:102A0000FF90EF90DF9008950F931F93CF93DF9384
:102A1000EC011A828CE391E0998388831B820091F8
:102A2000E5021091E60201151105F1F581E00E9421
:102A3000840D8C019093E6028093E502892BA1F529
:102A400063E070E081E00E94F90C9093E6028093CD
:102A5000E5021B8227E130E03E872D8725E230E04A
:102A60003C872B8727E430E0388B2F8728E030E045
:102A700038872F832AE230E03A872987009731F19F
:102A800068E00E9481068091E5029091E6026985E6
:102A900001960E9481068091E5029091E6026B8189
:102AA00002960E94810612C0C8010E947E1B90E01F
:102AB00098878F83C80101960E947E1B90E09A87B9
:102AC0008987C80102960E947E1B8B838B8181308F
:102AD00069F08230B1F087E190E09E878D8785E2D2
:102AE00090E09C878B8787E490E015C084E190E0BC
:102AF0009E878D8780E290E09C878B8785E390E0BE
:102B00000AC08EE190E09E878D8789E290E09C87E5
:102B10008B8789E490E0988B8F8789859A858038A8
:102B2000910524F08EE790E09A87898789859A85B8
:102B30002F813885821793071CF4019798878F831C
:102B400081E090E09D838C83DF91CF911F910F9165
:102B500008958091E7029091E802892BF9F480E0D2
:102B60000E94840D9093E8028093E702892BB1F4D0
:102B700062E070E080E00E94F90C9093E80280939C
:102B8000E702009759F061E00E9481068091E70218
:102B90009091E80260E001960C94810608950F93ED
:102BA0001F93CF93DF938C01EB01FC018381E881BC
:102BB000F981882359F00684F785E02DCB0109952A
:102BC000882309F4EAC0F8011382E7C00284F38580
:102BD000E02D64E070E0CE010995882381F083E068
:102BE00090E00E94001EFC0112822FE232E031834D
:102BF0002083BC01CE010E94BA0D80E017C0E8819D
:102C0000F9810284F385E02D61E070E0CE01099541
:102C1000882391F081E190E00E94001E8C010E94C7
:102C20000415B801CE010E94BA0D81E0DF91CF9169
:102C30001F910F910C94D512E881F9810284F385DC
:102C4000E02D6EE070E0CE0109958823D1F082E09E
:102C500090E00E94001E8C0187E192E0F8019183D0
:102C600080838C819D81009711F00E94981E1D83A6
:102C70000C838E819F819B838A831F821E8280E0CA
:102C800086C0E881F9810284F385E02D63E070E07D
:102C9000CE010995882369F088E190E00E94001E2A
:102CA0008C010E94400CB801CE010E94BA0D82E056
:102CB000BDCFE881F9810284F385E02D69E070E001
:102CC000CE0109958823D1F082E090E00E94001E99
:102CD0008C0189E292E0F801918380838C819D814F
:102CE000009711F00E94981E1D830C838E819F8196
:102CF0009B838A831F821E8281E049C0E881F9811B
:102D00000284F385E02D6AE070E0CE010995882306
:102D1000D1F082E090E00E94001E8C0183E292E0FC
:102D2000F801918380838C819D81009711F00E942E
:102D3000981E1D830C838E819F819B838A831F82B3
:102D40001E8282E024C0E881F9810284F385E02DAF
:102D50006BE070E0CE0109958823F9F082E090E005
:102D60000E94001E8C018DE192E0F8019183808326
:102D70008C819D81009711F00E94981E1D830C8309
:102D80008E819F819B838A831F821E8283E0DF91D5
:102D9000CF911F910F910C94C812DF91CF911F9189
:102DA0000F910895CF92DF92EF92FF920F931F93AE
:102DB000CF93DF936C017A018B01C0E0D0E0CE1598
:102DC000DF0581F0D8016D918D01D601ED91FC9167
:102DD0000190F081E02DC6010995892B11F0219613
:102DE000EECF7E01C701DF91CF911F910F91FF9030
:102DF000EF90DF90CF900895089580E090E00895DF
:102E0000FC01538D448D252F30E0842F90E0821BF0
:102E1000930B541710F0CF96089501970895FC0175
:102E2000918D828D981761F0828DDF01A80FB11D01
:102E30005D968C91928D9F5F9F73928F90E0089525
:102E40008FEF9FEF0895FC01918D828D981731F0DF
:102E5000828DE80FF11D858D90E008958FEF9FEF33
:102E600008950E94211F86E492E00E94930621E0CB
:102E7000892B09F420E0822F0895EF92FF920F939F
:102E80001F93CF93DF93EC0181E0888F9B8D8C8D16
:102E9000981305C0E889F989808185FD26C0F62E42
:102EA0000B8D10E00F5F1F4F0F731127E02E8C8DDD
:102EB000E8120CC00FB607FCFACFE889F9898081C7
:102EC00085FFF5CFCE010E941E0CF1CF8B8DFE0148
:102ED000E80FF11DE35AFF4FF0829FB7F8940B8F74
:102EE000EA89FB89808180620AC09FB7F894EE89E5
:102EF000FF896083E889F989808183708064808399
:102F00009FBF81E090E0DF91CF911F910F91FF90E3
:102F1000EF900895CF93DF93EC01888D8823C9F05B
:102F2000EA89FB89808185FD05C0A889B9898C91D2
:102F300086FD0FC00FB607FCF5CF808185FFF2CF6D
:102F4000A889B9898C9185FFEDCFCE010E941E0C16
:102F5000E7CFDF91CF9108951F920F920FB60F9296
:102F600011242F933F938F939F93AF93BF9380919F
:102F7000EF029091F002A091F102B091F202309133
:102F8000EE0223E0230F2D3720F40196A11DB11D81
:102F900005C026E8230F0296A11DB11D2093EE0265
:102FA0008093EF029093F002A093F102B093F202AB
:102FB00080913F0290914002A0914102B091420263
:102FC0000196A11DB11D80933F0290934002A093F2
:102FD0004102B0934202BF91AF919F918F913F9177
:102FE0002F910F900FBE0F901F9018951F920F9268
:102FF0000FB60F9211242F933F934F935F936F93CC
:103000007F938F939F93AF93BF93EF93FF9386E448
:1030100092E00E941E0CFF91EF91BF91AF919F91A2
:103020008F917F916F915F914F913F912F910F9071
:103030000FBE0F901F9018951F920F920FB60F9210
:1030400011242F938F939F93EF93FF93E091560258
:10305000F09157028081E0915C02F0915D0282FD67
:1030600012C0908180915F028F5F8F732091600208
:10307000821751F0E0915F02F0E0EA5BFD4F958F1F
:1030800080935F0201C08081FF91EF919F918F91AA
:103090002F910F900FBE0F901F901895E6E4F2E06D
:1030A0001382128288EE93E0A0E0B0E084839583DF
:1030B000A683B7838AE291E09183808385EC90E0D8
:1030C0009587848784EC90E09787868780EC90E0F2
:1030D000918B808B81EC90E0938B828B82EC90E0E3
:1030E000958B848B86EC90E0978B868B118E128E5D
:1030F000138E148E1092E4021092E3021092E602F4
:103100001092E5021092E8021092E7020895CF9320
:10311000DF9300D01F92CDB7DEB7789484B582607C
:1031200084BD84B5816084BD85B5826085BD85B56B
:10313000816085BD80916E00816080936E001092E9
:103140008100809181008260809381008091810064
:1031500081608093810080918000816080938000F5
:103160008091B10084608093B1008091B000816053
:103170008093B00080917A00846080937A0080917F
:103180007A00826080937A0080917A0081608093D7
:103190007A0080917A00806880937A001092C10052
:1031A000E0915602F091570282E08083E091520252
:1031B000F09153021082E0915402F091550280E1A7
:1031C000808310925E02E0915A02F0915B0286E0E9
:1031D0008083E0915802F091590280818061808360
:1031E000E0915802F0915902808188608083E091DB
:1031F0005802F0915902808180688083E0915802E2
:10320000F091590280818F7D80838091100190918F
:1032100011010197909311018093100143E050E058
:1032200062E070E0CE0101960E946E1B8981853AB2
:1032300031F48A818E3919F48B818C3811F080E059
:103240004DC089E090E00E947E1B8233A1F162E3D1
:1032500089E090E00E94810610924502109244029B
:1032600060E080E090E00E9481066091440281E08D
:1032700090E00E9481068091BE019091BF01A091D3
:10328000C00189839A83AB83CE0101967C0102E061
:1032900010E0D701DD907D01C8010E947E1BD81689
:1032A00021F06D2DC8010E94861B0F5F1F4F053056
:1032B000110579F712C080E090E00E947E1B90E03B
:1032C000909345028093440281E090E00E947E1B2F
:1032D00090E0909345028093440281E08093ED0258
:1032E0008BE491E00E94001E8C0185EC91E0F801D6
:1032F00091838083339681E2DF011D928A95E9F7FD
:10330000EB5BFE4F83E0DF011D928A95E9F7F80140
:1033100014A61093EC020093EB028CEB90E00E9459
:10332000001E21E032E0DC0111963C932E939C01BB
:103330002E583F4F1D963C932E931C9720E430E06F
:103340001B963C932E931A971E961C921E9791964D
:103350001C9291972AE0E3EFF1E0579601900D92CD
:103360002A95E1F79093EA028093E90283E00E94B4
:10337000571283E00E942F12F80112820E94A915B1
:103380008091E7029091E802009749F001960E942F
:103390007E1B823091F08330D1F0813039F082E0B1
:1033A00090E00E94001E27E132E00DC082E090E034
:1033B0000E94001E29E232E010C082E090E00E94EC
:1033C000001E23E232E0DC012D933C9309C082E031
:1033D00090E00E94001E2DE132E0FC013183208349
:1033E0006C010E94A9158091E7029091E802009774
:1033F00031F00E947E1B813081F08230B1F083E099
:1034000090E00E94001EDC0112961C9212972FE29F
:1034100032E02D933C938C010FC081E190E00E943B
:10342000001E8C010E94041507C088E190E00E94F4
:10343000001E8C010E94400CA090EB02B090EC02A8
:10344000E090E902F090EA0285E00E94571285E0E0
:103450000E942F1284E00E94571284E00E942F12D3
:10346000F701B186A08602831383C482D5821782B6
:10347000168235E3632E32E0732E5524539448E0D0
:10348000242E312C8091ED02882309F41CC18091F7
:10349000EB029091EC02DC01ED91FC910190F08146
:1034A000E02D09958111F7C00091E9021091EA021F
:1034B000F8018685C484D584A284B384882351F11D
:1034C000E12CF12CEA14FB0464F5C701F7FC079624
:1034D00023E0959587952A95E1F7F601E80FF91F06
:1034E0002081022E000C330BC701B1010E94D21DB6
:1034F00002C0359527958A95E2F7C9018170992711
:1035000020FF02C081E390E00E949E12FFEFEF1ABD
:10351000FF0AD8CF7601C7018C199D098A159B0532
:103520007CF08AE090E00E949E12D801ED91FC911F
:103530000484F585E02DC801099581110EC038C0BD
:10354000F70181917F01882319F081E390E002C0A7
:1035500080E090E00E949E12DECFD8011296ED919D
:10356000FC911397309719F08281811121C084E07A
:1035700090E00E94001E7C01FC01718260825382F7
:103580005282892B09F4A2C0F801868197810097A5
:1035900011F00E94981ED80112968D919C9113975C
:1035A00017969C938E9316971396FC92EE92129711
:1035B000C0901001D09011010D2C000CEE08FF08F6
:1035C0000E94A3124B015C01C114D104E104F10477
:1035D000F1F00E94A312DC01CB0188199909AA0914
:1035E000BB09883E9340A105B10570F3F1E0CF1A05
:1035F000D108E108F10828EE820E23E0921EA11CFA
:10360000B11CC114D104E104F10419F7DDCFF89421
:103610000091E9021091EA02D801ED91FC91048039
:10362000F581E02DC8010995F80180859185DC01BF
:10363000ED91FC910084F185E02D0995F8018281DE
:103640009381009751F040855185DC01ED91FC910B
:103650000190F081E02DB8010995F80186819781EC
:10366000892B71F484819581009751F040855185B3
:10367000DC01ED91FC910190F081E02DB8010995FC
:103680008091EB029091EC02DC01ED91FC910480C1
:10369000F581E02D09958091EB029091EC02DC011F
:1036A000ED91FC910280F381E02D0995F8948091D1
:1036B000EB029091EC02DC01ED91FC910680F78128
:1036C000E02D099578940E949F06DCCEF801868152
:1036D000978193838283178216826ACFDC01CB01A4
:1036E000FC01F999FECF06C0F2BDE1BDF89A319612
:1036F00000B40D9241505040B8F70895F999FECFAB
:1037000092BD81BDF89A992780B50895262FF99921
:10371000FECF1FBA92BD81BD20BD0FB6F894FA9AB4
:10372000F99A0FBE019608955058BB27AA270E9408
:10373000AC1B0C94261D0E94181D38F00E941F1D02
:1037400020F039F49F3F19F426F40C94151D0EF463
:10375000E095E7FB0C940F1DE92F0E94371D58F3ED
:10376000BA17620773078407950720F079F4A6F566
:103770000C94591D0EF4E0950B2EBA2FA02D0B01C1
:10378000B90190010C01CA01A0011124FF27591BA6
:1037900099F0593F50F4503E68F11A16F040A22FAC
:1037A000232F342F4427585FF3CF4695379527951D
:1037B000A795F0405395C9F77EF41F16BA0B620B1C
:1037C000730B840BBAF09150A1F0FF0FBB1F661F63
:1037D000771F881FC2F70EC0BA0F621F731F841FA6
:1037E00048F4879577956795B795F7959E3F08F0CC
:1037F000B0CF9395880F08F09927EE0F979587958E
:1038000008950E94EB1C08F481E008950E941A1CA0
:103810000C94261D0E941F1D58F00E94181D40F098
:1038200029F45F3F29F00C940F1D51110C945A1D7F
:103830000C94151D0E94371D68F39923B1F355238D
:1038400091F3951B550BBB27AA27621773078407B3
:1038500038F09F5F5F4F220F331F441FAA1FA9F349
:1038600035D00E2E3AF0E0E832D091505040E69537
:10387000001CCAF72BD0FE2F29D0660F771F881F98
:10388000BB1F261737074807AB07B0E809F0BB0B8B
:10389000802DBF01FF2793585F4F3AF09E3F51059F
:1038A00078F00C940F1D0C945A1D5F3FE4F3983E82
:1038B000D4F3869577956795B795F7959F5FC9F788
:1038C000880F911D9695879597F90895E1E0660F09
:1038D000771F881FBB1F621773078407BA0720F082
:1038E000621B730B840BBA0BEE1F88F7E0950895EB
:1038F0000E947F1C6894B1110C945A1D08950E9477
:103900003F1D88F09F5798F0B92F9927B751B0F015
:10391000E1F0660F771F881F991F1AF0BA95C9F753
:1039200014C0B13091F00E94591DB1E008950C947B
:10393000591D672F782F8827B85F39F0B93FCCF32E
:10394000869577956795B395D9F73EF490958095D0
:10395000709561957F4F8F4F9F4F0895E89409C0F0
:1039600097FB3EF490958095709561957F4F8F4FB2
:103970009F4F9923A9F0F92F96E9BB279395F695C8
:10398000879577956795B795F111F8CFFAF4BB0F46
:1039900011F460FF1BC06F5F7F4F8F4F9F4F16C0AA
:1039A000882311F096E911C0772321F09EE8872F34
:1039B000762F05C0662371F096E8862F70E060E0F0
:1039C0002AF09A95660F771F881FDAF7880F969569
:1039D000879597F90895990F0008550FAA0BE0E80D
:1039E000FEEF16161706E807F907C0F012161306C1
:1039F000E407F50798F0621B730B840B950B39F401
:103A00000A2661F0232B242B252B21F408950A2666
:103A100009F4A140A6958FEF811D811D089597F9A6
:103A20009F6780E870E060E008959FEF80EC089564
:103A300000240A941616170618060906089500248D
:103A40000A9412161306140605060895092E039407
:103A5000000C11F4882352F0BB0F40F4BF2B11F47B
:103A600060FF04C06F5F7F4F8F4F9F4F089557FDDA
:103A70009058440F551F59F05F3F71F04795880FDC
:103A800097FB991F61F09F3F79F087950895121673
:103A900013061406551FF2CF4695F1DF08C016161F
:103AA00017061806991FF1CF8695710561050894D0
:103AB0000895E894BB2766277727CB0197F90895E7
:103AC0000E94EB1C08F48FEF08950E94781D0C945F
:103AD000261D0E94181D38F00E941F1D20F09523FE
:103AE00011F00C940F1D0C94151D11240C945A1DEB
:103AF0000E94371D70F3959FC1F3950F50E0551F3D
:103B0000629FF001729FBB27F00DB11D639FAA2732
:103B1000F00DB11DAA1F649F6627B00DA11D661F81
:103B2000829F2227B00DA11D621F739FB00DA11DA2
:103B3000621F839FA00D611D221F749F3327A00D5C
:103B4000611D231F849F600D211D822F762F6A2FF8
:103B500011249F5750409AF0F1F088234AF0EE0F5D
:103B6000FF1FBB1F661F771F881F91505040A9F78A
:103B70009E3F510580F00C940F1D0C945A1D5F3F21
:103B8000E4F3983ED4F3869577956795B795F795C6
:103B9000E7959F5FC1F7FE2B880F911D969587953E
:103BA00097F9089597FB072E16F4009407D077FD38
:103BB00009D00E94E61D07FC05D03EF49095819542
:103BC0009F4F0895709561957F4F0895AA1BBB1B69
:103BD00051E107C0AA1FBB1FA617B70710F0A61B0D
:103BE000B70B881F991F5A95A9F780959095BC012E
:103BF000CD010895EE0FFF1F0590F491E02D09947B
:103C00000F931F93CF93DF938230910510F482E0DE
:103C100090E0E091F502F091F60220E030E0A0E0C3
:103C2000B0E0309719F1408151810281138148172A
:103C30005907C8F08417950769F4109731F0129668
:103C40000C93129713961C9327C00093F5021093C0
:103C5000F60222C02115310519F04217530718F456
:103C60009A01BD01EF01DF01F801DBCF211531051C
:103C7000F9F0281B390B2430310580F48A819B81AF
:103C80006115710521F0FB019383828304C0909339
:103C9000F6028093F502FE01329644C0FE01E20F67
:103CA000F31F8193919322503109398328833AC0BD
:103CB0002091F3023091F402232B41F4209114015E
:103CC000309115013093F4022093F30220911201F8
:103CD000309113012115310541F42DB73EB74091C4
:103CE000160150911701241B350BE091F302F0915E
:103CF000F402E217F307A0F42E1B3F0B2817390735
:103D000078F0AC014E5F5F4F2417350748F04E0F37
:103D10005F1F5093F4024093F3028193919302C08A
:103D2000E0E0F0E0CF01DF91CF911F910F91089576
:103D3000CF93DF93009709F481C0FC01329713827F
:103D40001282A091F502B091F602109781F42081C1
:103D50003181820F931F2091F3023091F4022817D2
:103D6000390751F5F093F402E093F30267C0ED01D7
:103D700020E030E0CE17DF0740F44A815B819E01EE
:103D800041155105F1F0EA01F5CFD383C28340819B
:103D90005181840F951FC817D90759F488819981DB
:103DA000840F951F0296918380838A819B819383E0
:103DB00082832115310529F4F093F602E093F50290
:103DC0003DC0E901FB83EA8349915991C40FD51F96
:103DD000EC17FD0761F480819181840F951F029695
:103DE000E90199838883828193819B838A83E0E0C0
:103DF000F0E012968D919C911397009719F0FD01B8
:103E0000DC01F7CF8D919C9111979D012E5F3F4F63
:103E1000820F931F2091F3023091F4022817390783
:103E200069F4309729F41092F6021092F50202C05C
:103E300013821282B093F402A093F302DF91CF9128
:103E4000089581E090E0F8940C942D1FDC0101C0EE
:0E3E50006D9341505040E0F70895F894FFCF75
:103E5E0009000300000000000101400300400301BF
:103E6E000C000000F702800000807F7F7F7F000043
:103E7E00000000007C07000000003D17D21600175E
:103E8E008A1793060F17231700000000DF12001089
:103E9E00111213141516171718191A1B1B1C1D1E99
:103EAE001E1F2021222223242425262627282829C6
:103EBE002A2A2B2C2C2D2D2E2F2F30303131323310
:103ECE0033343435353636373738383839393A3A77
:103EDE003B3B3B3C3C3D3D3D3E3E3F3F3F404040FB
:103EEE00404141414242424343434343444444449C
:103EFE00444545454545464646464646464646465B
:103F0E004747474747474747474747474747A59E7E
:103F1E008C00000000F806F5061A0C860B71076778
:103F2E00075F07510745070107FB0606070000005C
:103F3E0000000000003117311731173117311731DA
:103F4E001731170080808080800000020200000080
:103F5E0000F80C840BBE09ED06E506C806BC06B2D9
:103F6E0006A90600000000230300000000870000E1
:103F7E00000000D50100000000A704000000007141
:0E3F8E000400000000CF1500000000311700F5
:00000001FF
